:020000040000FA
:0400000006EF02F015
:08000800E8CF05F0D8CF06F0A7
:10001000E0CF07F00001E9CF0DF0EACF08F0E1CF23
:1000200009F0E2CF0AF0D9CF0BF0DACF0CF0F3CF22
:1000300014F0F4CF15F0FACF16F000C00FF001C0A5
:1000400010F002C011F003C012F004C013F09DAA1A
:100050002DEF00F09EBA9EEF00F00FC000F010C030
:1000600001F011C002F012C003F013C004F00DC083
:10007000E9FF08C0EAFF09C0E1FF0AC0E2FF0BC0C8
:10008000D9FF0CC0DAFF14C0F3FF15C0F4FF16C08F
:10009000FAFF05C0E8FF07C0E0FF06C0D8FF100068
:1000A000F2CF0EF0F29EF76ABA0FF66E000EF7224C
:1000B0000900F5500EBEF28E12000A0D496E6974E9
:1000C00069616C697A696E6720506F727420420AA8
:1000D0000D00F2CF0EF0F29EF76AEC0FF66E000EF6
:1000E000F7220900F5500EBEF28E1200436F6E66C5
:1000F00069677572696E672052462D3234470A0D62
:100100000000F2CF0EF0F29EF76A1C0FF66E010EA1
:10011000F7220900F5500EBEF28E12004F4B210A55
:100120000D0A0D009EAAFED7ABCF18F0AECF01F09E
:1001300018A202D0AB98AB880000000CF3DF01C01E
:1001400027F02750120A03E0770A26E039D0EADFC9
:100150000150340802E0000E01D0010E296EE2DFEA
:100160000150560802E0000E01D0010E29142B6E3A
:10017000D9DF0150780802E0000E01D0010E2B14E7
:100180002D6ED0DF0150900802E0000E01D0010E6C
:100190002D14D8A4FF0014D0C5DF01C019F0C2DFB0
:1001A00001C01AF0BFDF01C01BF0BCDF01C01CF0B2
:1001B000B9DF01C01DF0B6DF01C01EF01F8000D006
:1001C0009E9A2DEF00F0EA6A200EE96EEF500FE0E4
:1001D000030E016E006A002EFED7012EFBD73C0EE7
:1001E000006E002EFED700000000EF2EF1D7000CAD
:1001F000070E246E236A235007081DE3939A8A9AF8
:1002000024502406256E22C000F02550016E04E023
:10021000D8900032012EFCD700A003D093988A8892
:1002200002D093988A9800000000939A8A8A00006E
:100230000000232AE0D7000C93968A96939E8A9E0C
:10024000939A8A9A93988A98030E206EBCDF939EA5
:100250008A8E080E006E002EFED7300E226EC8DF8A
:10026000300E226EC5DF226AC3DF226AC1DF226A36
:10027000BFDF420E226EBCDF420E226EB9DF226A61
:10028000B7DF226AB5DF226AB3DF420E226EB0DF2B
:10029000420E226EADDF430E226EAADF6F0E226E7B
:1002A000A7DF810E226EA4DF938893968A96939E91
:1002B0008A9E939A8A9A75EF02F093968A96939EF5
:1002C0008A8E080E006E002EFED793988A88939A25
:1002D0008A8A00000000939A8A9A00000000939E88
:1002E0008A9E9388939A8A9A93968A86000C246AA7
:1002F000070E256E236A235007082BE3939A8A9AE8
:1003000000000000939A8A8A00000000938881A868
:100310000FD025502506266E010E006E2650016E68
:1003200004E0D8900036012EFCD7005024120FD0E4
:1003300025502506266E010E006E2650016E04E043
:10034000D8900036012EFCD70050FF0A2416232A2D
:10035000D2D724C001F0BCEF01F0206A205005087C
:1003600013E3036A2050190F016E000E032201C02F
:1003700021F003C022F0BBD722C0EAFF21C0E9FF71
:1003800001C0EFFF202AEAD7939A8A9A93968A8629
:100390008DEF02F093968A96939E8A8E080E006ED9
:1003A000002EFED793988A98939A8A8A00000000BC
:1003B000939A8A9A00000000939E8A9E939A8A9A42
:1003C000ACEF02F093968A86080E006E002EFED7E0
:1003D000420E226E0DDF420E226E0ADF206A20508E
:1003E00005080EE3036A2050190FE96E000E032082
:1003F000EA6EEFCF21F021C022F0FADE202AEFD7FB
:1004000093968A96939A8A9AB0EF02F0F86AD09EF1
:100410000D8EEA6AE96AB8862A0EAF6E000EB06EDB
:10042000260EAC6E900EAB6EC150C00B0F09C16EA4
:10043000070EB46E186A1F90C150C00B0F09C16E31
:10044000C290880ED56ECD6A000ECA6E7F0ECB6E3E
:10045000B150480BB16EB70EB1169484BD6ABD6A37
:10046000B1169482BA6ABA6A9D8AC00EF212640EFC
:10047000206EA9DE206A205013DE202A006E005074
:100480009EA8FED7AD6E150E205CF5E1030E216E21
:100490002E0E9EA8FED7AD6E212EFAD70A0E9EA86C
:1004A000FED7AD6E0D0E9EA8FED7AD6EF18EF29604
:1004B000206A20500EDE202A006E00509EA8FED733
:1004C000AD6E120E205CF5E1030E216E2E0E9EA87D
:1004D000FED7AD6E212EFAD70A0E9EA8FED7AD6EBE
:1004E0000D0E9EA8FED7AD6EA7D6E7DE7F0E196E65
:1004F0001A6E1B6E1C6E1D6E1E6E206A205001DE71
:10050000202A006E00509EA8FED7AD6E070E205C1C
:10051000F5E1938C81AC1DD020D7650E9EA8FED747
:10052000AD6E19509EA8FED7AD6E1A509EA8FED78C
:10053000AD6E1B509EA8FED7AD6E1C509EA8FED778
:10054000AD6E1D509EA8FED7AD6E1E509EA8FED764
:10055000AD6E1FA00DD01ED7010E206E34DE32D737
:10056000010E206E30DEA9DE010E206E2CDE1F9003
:04057000D0D70300DD
:00000001FF
